:100000000C94A70D0C94C30D0C94C30D0C94C30D4C
:100010000C94C30D0C94C30D0C94C30D0C94C30D20
:100020000C94C30D0C94C30D0C94C30D0C94C3130A
:100030000C94C30D0C94C30D0C94C30D0C94C30D00
:100040000C94C30D0C94C30D0C94F20D0C94C30DC1
:100050000C94C30D0C94C30D0C94C30D0C94C30DE0
:100060000C94C30D0C94C30D0C94C30D0C94C30DD0
:100070000C94C30D1201000209000108AAAACCCCFD
:1000800000010000000109021900010100E032092D
:1000900004000001090000000705810301000C09AC
:1000A0002906A900326400FF1201000200000008C6
:1000B000AAAA55550000000000040902000F010023
:1000C00000801201000200000008AAAABBBB0000C9
:1000D000000000010902160001010080010904006E
:1000E0000000FE0102000421B42F120100020000F2
:1000F0000008AAAA555500000000000209024D0A96
:1001000001010080010904000000FE010200090451
:10011000000000FE0102000904000000FE010200D0
:100120000904000000FE0102000904000000FE01B5
:1001300002000904000000FE010200090009040099
:100140000000FE0102000904000000FE0102000997
:1001500004000000FE0102000904000000FE01028C
:10016000000904000000FE0102000904000000FE76
:100170000102000904000000FE010200020009045F
:10018000000000FE0102000904000000FE01020060
:100190000904000000FE0102000904000000FE0145
:1001A00002000904000000FE010200090400000032
:1001B000FE0102000904000000FE01020102000924
:1001C00004000000FE0102000904000000FE01021C
:1001D000000904000000FE0102000904000000FE06
:1001E0000102000904000000FE01020009040000F1
:1001F00000FE0102000904000000FE01FE010200F1
:100200000904000000FE0102000904000000FE01D4
:1002100002000904000000FE0102000904000000C1
:10022000FE0102000904000000FE010200090400B2
:100230000000FE0102000904000000FE00FE0102B1
:10024000000904000000FE0102000904000000FE95
:100250000102000904000000FE0102000904000080
:1002600000FE0102000904000000FE010200090472
:10027000000000FE01020009040000000000FE0171
:1002800002000904000000FE010200090400000051
:10029000FE0102000904000000FE01020009040042
:1002A0000000FE0102000904000000FE0102000936
:1002B00004000000FE01020009040000000000FE2E
:1002C0000102000904000000FE0102000904000010
:1002D00000FE0102000904000000FE010200090402
:1002E000000000FE0102000904000000FE010200FF
:1002F0000904000000FE01020009040004000000DF
:10030000FE0102000904000000FE010200090400D1
:100310000000FE0102000904000000FE01020009C5
:1003200004000000FE0102000904000000FE0102BA
:10033000000904000000FE01020009040904000095
:1003400000FE0102000904000000FE010200090491
:10035000000000FE0102000904000000FE0102008E
:100360000904000000FE0102000904000000FE0173
:1003700002000904000000FE010200090009040057
:100380000000FE0102000904000000FE0102000955
:1003900004000000FE0102000904000000FE01024A
:1003A000000904000000FE0102000904000000FE34
:1003B0000102000904000000FE010200020009041D
:1003C000000000FE0102000904000000FE0102001E
:1003D0000904000000FE0102000904000000FE0103
:1003E00002000904000000FE0102000904000000F0
:1003F000FE0102000904000000FE010201020009E2
:1004000004000000FE0102000904000000FE0102D9
:10041000000904000000FE0102000904000000FEC3
:100420000102000904000000FE01020009040000AE
:1004300000FE0102000904000000FE01FE010200AE
:100440000904000000FE0102000904000000FE0192
:1004500002000904000000FE01020009040000007F
:10046000FE0102000904000000FE01020009040070
:100470000000FE0102000904000000FE00FE01026F
:10048000000904000000FE0102000904000000FE53
:100490000102000904000000FE010200090400003E
:1004A00000FE0102000904000000FE010200090430
:1004B000000000FE01020009040000000000FE012F
:1004C00002000904000000FE01020009040000000F
:1004D000FE0102000904000000FE01020009040000
:1004E0000000FE0102000904000000FE01020009F4
:1004F00004000000FE01020009040000000000FEEC
:100500000102000904000000FE01020009040000CD
:1005100000FE0102000904000000FE0102000904BF
:10052000000000FE0102000904000000FE010200BC
:100530000904000000FE010200090400040000009C
:10054000FE0102000904000000FE0102000904008F
:100550000000FE0102000904000000FE0102000983
:1005600004000000FE0102000904000000FE010278
:10057000000904000000FE01020009040904000053
:1005800000FE0102000904000000FE01020009044F
:10059000000000FE0102000904000000FE0102004C
:1005A0000904000000FE0102000904000000FE0131
:1005B00002000904000000FE010200090009040015
:1005C0000000FE0102000904000000FE0102000913
:1005D00004000000FE0102000904000000FE010208
:1005E000000904000000FE0102000904000000FEF2
:1005F0000102000904000000FE01020002000904DB
:10060000000000FE0102000904000000FE010200DB
:100610000904000000FE0102000904000000FE01C0
:1006200002000904000000FE0102000904000000AD
:10063000FE0102000904000000FE0102010200099F
:1006400004000000FE0102000904000000FE010297
:10065000000904000000FE0102000904000000FE81
:100660000102000904000000FE010200090400006C
:1006700000FE0102000904000000FE01FE0102006C
:100680000904000000FE0102000904000000FE0150
:1006900002000904000000FE01020009040000003D
:1006A000FE0102000904000000FE0102000904002E
:1006B0000000FE0102000904000000FE00FE01022D
:1006C000000904000000FE0102000904000000FE11
:1006D0000102000904000000FE01020009040000FC
:1006E00000FE0102000904000000FE0102000904EE
:1006F000000000FE01020009040000000000FE01ED
:1007000002000904000000FE0102000904000000CC
:10071000FE0102000904000000FE010200090400BD
:100720000000FE0102000904000000FE01020009B1
:1007300004000000FE01020009040000000000FEA9
:100740000102000904000000FE010200090400008B
:1007500000FE0102000904000000FE01020009047D
:10076000000000FE0102000904000000FE0102007A
:100770000904000000FE010200090400040000005A
:10078000FE0102000904000000FE0102000904004D
:100790000000FE0102000904000000FE0102000941
:1007A00004000000FE0102000904000000FE010236
:1007B000000904000000FE01020009040904000011
:1007C00000FE0102000904000000FE01020009040D
:1007D000000000FE0102000904000000FE0102000A
:1007E0000904000000FE0102000904000000FE01EF
:1007F00002000904000000FE0102000900090400D3
:100800000000FE0102000904000000FE01020009D0
:1008100004000000FE0102000904000000FE0102C5
:10082000000904000000FE0102000904000000FEAF
:100830000102000904000000FE0102000200090498
:10084000000000FE0102000904000000FE01020099
:100850000904000000FE0102000904000000FE017E
:1008600002000904000000FE01020009040000006B
:10087000FE0102000904000000FE0102010200095D
:1008800004000000FE0102000904000000FE010255
:10089000000904000000FE0102000904000000FE3F
:1008A0000102000904000000FE010200090400002A
:1008B00000FE0102000904000000FE01FE0102002A
:1008C0000904000000FE0102000904000000FE010E
:1008D00002000904000000FE0102000904000000FB
:1008E000FE0102000904000000FE010200090400EC
:1008F0000000FE0102000904000000FE00FE0102EB
:10090000000904000000FE0102000904000000FECE
:100910000102000904000000FE01020009040000B9
:1009200000FE0102000904000000FE0102000904AB
:10093000000000FE01020009040000000000FE01AA
:1009400002000904000000FE01020009040000008A
:10095000FE0102000904000000FE0102000904007B
:100960000000FE0102000904000000FE010200096F
:1009700004000000FE01020009040000000000FE67
:100980000102000904000000FE0102000904000049
:1009900000FE0102000904000000FE01020009043B
:1009A000000000FE0102000904000000FE01020038
:1009B0000904000000FE0102000904000400000018
:1009C000FE0102000904000000FE0102000904000B
:1009D0000000FE0102000904000000FE01020009FF
:1009E00004000000FE0102000904000000FE0102F4
:1009F000000904000000FE010200090409040000CF
:100A000000FE0102000904000000FE0102000904CA
:100A1000000000FE0102000904000000FE010200C7
:100A20000904000000FE0102000904000000FE01AC
:100A300002000904000000FE010200090009040090
:100A40000000FE0102000904000000FE010200098E
:100A500004000000FE0102000904000000FE010283
:100A6000000904000000FE0102000904000000FE6D
:100A70000102000904000000FE0102000200090456
:100A8000000000FE0102000904000000FE01020057
:100A90000904000000FE0102000904000000FE013C
:100AA00002000904000000FE010200090400000029
:100AB000FE0102000904000000FE0102010200091B
:100AC00004000000FE0102000904000000FE010213
:100AD000000904000000FE0102000904000000FEFD
:100AE0000102000904000000FE01020009040000E8
:100AF00000FE0102000904000000FE01FE010200E8
:100B00000904000000FE0102000904000000FE01CB
:100B100002000904000000FE0102000904000000B8
:100B2000FE0102000904000000FE010200090400A9
:100B30000000FE0102000904000000FE00FE0102A8
:100B4000000904000000FE01021201000200000082
:100B500008AAAA555500000000000309021200016E
:100B6000010080010904000000FE010200090212D8
:100B70000001010080090200000101008001090458
:100B8000000000FE010200090230000101008001A6
:100B90000904000000FE0102003E2100000000FAEE
:100BA000CEB003AABBCCDD80000000004650008020
:100BB000000000003DEE7012010002000000084C31
:100BC00005EB020000000000010902200001000006
:100BD00080010904000002FF00000007050202086E
:100BE0000000070581020800001201000200000059
:100BF00008AAAAC0DE0000000000010902120001DC
:100C0000010080010904000000FE01020009021237
:100C10000001000080FA0904000000FE010200004B
:100C20000000000000FACEB003AABBCCDD3863F0B0
:100C30000038A01000388000017884F80664840031
:100C40007F6084EE2838A5FFF87CC3282A7CC4295D
:100C50002A282500004082FFF0388400587C890350
:100C6000A64E8004207C0802A6F821FF61FB6100EB
:100C700078FB810080FBA10088FBC10090FBE100B4
:100C800098F80100B03BE000017BFFF8067FE3FB32
:100C9000786463007F6063F0204B8D34257FE4FB34
:100CA000786484002E6084B1287FE3FB786463005D
:100CB0007F6063F010F86401207FE5FB7864A50095
:100CC0007F60A5EF3C8065000028030000418200A2
:100CD00018808500047C63FA149083000038A50016
:100CE000084BFFFFE4EB610078EB810080EBA10093
:100CF00088EBC10090EBE10098E80100B0382100DA
:100D0000A07C0803A6386000017863F806646300DD
:100D10007F6063EE283880000038A001D84B84E261
:100D20000C000490E0E8820F08000490E4E87C00E6
:100D300020000490E8F86400000004F0A8487B025A
:100D400085002AAFF0485541FC0004ED18388000BA
:100D5000000004ED1C908300000004ED204E800094
:100D600020003BA89001000000000505D0487AF063
:100D7000FC000234D0487DC1CD000E83D44871728E
:100D8000C90004F2904BFFFFD40005739860000087
:100D90000000057408480000A00005745C3BE000FA
:100DA0000000017CBCE863000000017CC04E8000B4
:100DB0002000017CC8F883000000017CCC4E80003C
:100DC0002000017CD4487E781000050B3C38600080
:100DD0000100050B404E80002000000000000000D4
:100DE0000000000000386000014E800020386000E4
:100DF000004E80002080000000007FF15080000045
:100E0000000033E72080000000007FF81A80000017
:100E100000007FF04080000000007FF05080000064
:100E200000007FF06080000000007FF08080000004
:100E3000000033E72080000000007FF0C880000041
:100E4000000033E72080000000007FF124800000D4
:100E5000000033E72080000000007FF12C800000BC
:100E6000000033E720F821FF817C0802A6F801008A
:100E7000903880000038A000014B8D390580A30018
:100E800008386000003C80AAAA6084C0DE7C042888
:100E900040418200083860FFFF7C6307B4E801002E
:100EA000907C0803A6382100804E800020F821FFA6
:100EB000817C0802A6F8010090388000004B8D3834
:100EC000ED3881007038A00000F8A4000038C0217F
:100ED000AAB0C4000038C00000B0C4000638C0008A
:100EE0000178C6F80664C6007F60C6F07038E0007E
:100EF000004B8D382138600000E80100907C080329
:100F0000A6382100804E800020386000004E80000E
:100F1000202C0300004082001C386000017863F838
:100F2000066463007F6063F7CC3880000190830023
:100F3000104E800020F821FF317C0802A6F8010045
:100F4000E0FBE100C8388100704B9B49D93BE000D1
:100F5000017BFFF8063880000267E3007F6063F7DB
:100F6000849083000067FF007F63FFF7CCE87F0079
:100F7000002C2300004182000C388000274B863370
:100F80003138800027386008004B862EE5F87F0056
:100F900000E88100704B84E141E861007038800016
:100FA000274B86330DE87F00004B84E155E89F0016
:100FB000007C641A14F87F000838600000EBE10040
:100FC000C8E80100E0382100D07C0803A64E80006C
:100FD000203BE000017BFFF80667FB007F637BF7A7
:100FE000E4EB5B0000283A00004182004C7FA3EB59
:100FF00078E89A0000282400004182003C80BA0072
:10100000104B84E129282300004082002480BA008C
:10101000107C9D2A14E87A00087C7D1B7880BA0039
:10102000147C632A144B84E0B1480000D83B5A007A
:10103000184BFFFFBC67E4007F6084F82638A000EF
:10104000094B84E0E9282300004082006867FA0029
:101050007F635AF81EEB7A0000283B0000408200B4
:101060002438800027386008004B862E05F87A0067
:10107000007C7B1B7867E4007F6084F8304B84E061
:1010800059387B000B67E5007F60A5F7CCE8850049
:1010900000282400004182000C7C9B2378E8650036
:1010A00008389D00094B84E0317F7DDB7841820068
:1010B000547FA3EB787FE4FB786484007F6084F83E
:1010C0001038A000094B84E065282300004082000E
:1010D0003467FF007F63FFF7CC807F001028030098
:1010E0000041820020E87F000028230000418200A8
:1010F00014E87F0008389D00094B84DFDDEBBF005A
:10110000007F84E3787FA3EB784B84DFF54BAABCA8
:10111000CC7C0802A6F821FE61FB610078FB81000F
:1011200080FBA10088FBC10090FBE10098F8010161
:10113000B07C7D1B787C9E23783BE000017BFFF830
:1011400006EB829600EB9C0068EB9C0018EB620FAC
:1011500008E93D001881290030792984022C090012
:101160002940820058E89C00107885C1E478A546A3
:10117000202C0500FF4182001860840003F89C00C9
:101180001038600006907E00004800001460840063
:1011900002F89C00103860002C907E000080BC009B
:1011A00004E89C0008E87B00007D232A14F93B003A
:1011B000004B87CC51480000EC7FA3EB787FC4F351
:1011C000784B84F4417FFDFB7867BD007F63BDF7FA
:1011D000E0807D000080BC00047C632A14907D00C8
:1011E00000E89C00107885C1E478A546202C050015
:1011F000FF408200B0E87B00003880000038C0006B
:10120000007CE3221480A700007CC62A7838840082
:1012100004282404004082FFEC807D000078C6078B
:10122000C67CC61B7838600000907D00007FE7FB1D
:101230007864E7007F60E7F6F4E8670000282300A1
:10124000004182006038E700107C2330404082FF7C
:10125000ECE8A7FFF8E8FB00008065000028030029
:101260000041820040280300014182002028030041
:101270000241820028808500047C633A1490830038
:101280000038A500084BFFFFD4806500047CA51A38
:101290001438A500084BFFFFC438A500084BFFFF1A
:1012A000BC38600000EB610078EB810080EBA100AE
:1012B00088EBC10090EBE10098E80101B038210112
:1012C000A07C0803A64E8000207C0802A6F821FF1F
:1012D00061FB610078FB810080FBA10088FBC100FD
:1012E00090FBE10098F80100B03BE000017BFFF8C3
:1012F0000667FB007F637BF7EC839B0000281C00E4
:10130000004182006C281C0008408000B82823009F
:1013100001408200B0282400004182000C3B9C0068
:1013200001939B0000EB9B00087C24E0404082007E
:10133000943B800001939B000067E4002E6084B121
:1013400028EB9B0010FB840030EB9B0018FB840013
:101350003867FC007F639CF010FB8401203B800019
:1013600000939B0000386001004800003470630067
:10137000FF2823000A4080005867FB007F637BF84A
:101380003C787C1F247F7BE214EBBB00007C832332
:10139000787CA42B787CC533784800003DEB610055
:1013A00078EB810080EBA10088EBC10090EBE100BD
:1013B00098E80100B0382100A07C0803A64E800008
:1013C000203C608001606300034BFFFFD43860FF66
:1013D000FF4BFFFFCC7FA903A64E80042067FB00D4
:1013E0007F637BF7ECF87B00083B800001939B0058
:1013F0000067E4002E6084B128E8640128EB8400D3
:1014000030F8640030FB9B0010EB840038F8640077
:1014100038FB9B0018F8640120386000004E800003
:1014200020386001004E8000204B87C9D84B84DAF9
:10143000FC7C6903A67C8323787CA42B784E8004F3
:10144000204B862A2C4B862E6838600000396000BD
:10145000FF4400002267FB007F637BF80C907B0059
:1014600000386000004E8000207C641B7867FB0021
:101470007F637BF7E4E87B0000F89B00004E800070
:1014800020392000017929F8066529007F6129F8B3
:101490000C80090000280000014182F94C2800005E
:1014A000024182F94CE92296887C0802A64B850FFE
:1014B00010392000017929F8066529007F6129F893
:1014C0000C80090000280000004082F91CE92296E7
:1014D000887C0802A64B850EE8A0556F3D002CB80D
:1014E000FD80000000007FF73C8C0A948C000D9971
:1014F000B180000000007FF764A2BC1A5600052AE4
:10150000DC80000000007FF7A86B7028020002005A
:101510001780000000007FF7580000000000000066
:10152000000030535438600082005F3FC0386000D4
:1015300001005F3FC44E800020000000000002EE6A
:10154000F060000000000000000022B8885F746FA7
:101550006F0022B88C6C322E780022B8906D6C230C
:10156000720022B8946F6F74000000000100000048
:1015700018002367E82F646576002367EC5F6264D8
:1015800076002367F0642F505300000000000D68C0
:10159000B85F746F6F000D68BC6C322E78000D68F8
:1015A000C06D6C2372000D68C46F6F740000000082
:1015B000000000000000000000000000000000002B
:1015C000000000000000000000000000000000001B
:1015D000000000000000000000000000000000000B
:1015E00000000000000000000000000000000000FB
:1015F00000000000022F6465765F62647664006D0F
:101600006F640000000000000000002F6170705F38
:10161000686F6D65002F6465765F7573623030307A
:101620000080000000007FF5F880000000007FF6D9
:101630003C80000000007FF64480000000007FF640
:101640004880000000007FF64C80000000007FF61C
:101650005C80000000007FF66080000000007FF6E4
:101660006480000000007FF67080000000007FF6BC
:101670008480000000007FF63C00000000000000B5
:10168000000000000000000000000000000000005A
:10169000000000000000000000000000000000004A
:1016A000000000000000000000000000000000003A
:1016B000000000000000000000000000000000002A
:101B00000000000000000000000000000080000055
:101B100000003DEE7880000000003DEE888000006F
:101B2000000033E720E883FFF0E863FFF8E8A30054
:101B300018386310007C0428004082FFF438C3F09A
:101B4000207CC903A64E800420040000000011245C
:101B50001FBECFEFD2E0DEBFCDBF11E0A0E0B1E00D
:101B6000E0EEFCE202C005900D92A431B107D9F776
:101B700011E0A4E1B1E001C01D92A933B107E1F782
:101B80005CD30C946E160C940000E0911301FF27B7
:101B9000E7FDF095E45FFE4F8F778083E3EEF0E0A2
:101BA00080838081806880830895982F80911301BD
:101BB0008917B9F090931301E92FFF27E7FDF095FE
:101BC000DF01A45FBE4F8C9187FD1C92E45FFE4F46
:101BD00080818F778093E3008091E3008068809319
:101BE000E30008951F920F920FB60F9211248F9366
:101BF00086EF809385008CE3809384008091270199
:101C0000882329F0809127018150809327018F91AB
:101C10000F900FBE0F901F90189528EE33E0782F8D
:101C2000709540E951E0609505C0CA010197F1F750
:101C30002150304021153105C1F78BB180648723D5
:101C40008BB988EE93E0FA013197F1F70197D9F754
:101C50008BB1806486238BB928EE33E0E6CF81E038
:101C60008093E9008091E80085FF18C090912101E0
:101C70009923A1F080912201882339F08091EB0013
:101C800088608093EB00109222019093F100809184
:101C9000E8008E778093E800109221010895FC01FE
:101CA000109226011092250121E030E0C9010E2E8C
:101CB00002C0880F991F0A94E2F78093210131979F
:101CC000EE0FFF1FDF01A050BF4F83E091E08D9327
:101CD0009C93EC5EFE4F318320830895FC011092AB
:101CE00024011092230121E030E0C9010E2E02C030
:101CF000880F991F0A94E2F7809321013197EE0F24
:101D0000FF1FDF01A050BF4F80E091E08D939C93B7
:101D1000EC5EFE4F318320830895FA016091370114
:101D200070913801923081F1993209F4AEC091304E
:101D300009F0B4C0809113018330D1F084303CF4B9
:101D4000813081F082308CF4882349F0A7C085303F
:101D5000A9F0853084F0863009F0A0C012C044E7B5
:101D600050E06BC048EA50E068C042EC50E065C00B
:101D70004AEE50E062C049E45BE05FC047EB5BE0E5
:101D80005CC049EE5BE059C090911301933009F4B7
:101D900040C094303CF49130A1F092307CF599230E
:101DA00059F07CC0953009F468C095300CF441C0FE
:101DB000963009F073C066C046E850E029E130E093
:101DC00071C0843008F06AC06830710529F04DE0B8
:101DD0005CE020E03FE004C04AEB50E028E030E067
:101DE000833009F05FC06930710508F45BC085E09D
:101DF000809320018AE08093270154C088E080937B
:101E000020018FE08093270144ED50E026E130E08F
:101E100049C0813049F46930710530F08BE080931E
:101E200020018AE0809327014CEF50E02DE43AE056
:101E300039C0882329F44BE55BE022E130E032C071
:101E4000813059F46830710519F045E75BE0F5CF52
:101E50004DE65BE028E030E025C08230F9F46930DF
:101E6000710530F080E18093200184E180932701A7
:101E700047E85BE020E330E015C049EC5BE020E29E
:101E800030E010C04BEF5BE0D8CF80911301882386
:101E900029F44FE950E029E030E004C040E050E090
:101EA00020E030E051834083C901089508950895EA
:101EB0000895089581E061EC42E045D3882329F438
:101EC00080E090E060E470E0A8DE82E060EC42E058
:101ED0003AD3882329F480E090E060E470E09DCE5E
:101EE00008951F93809113018630A1F480913201EF
:101EF0008A3A09F023C18091E800877F8093E80047
:101F00008091E8008E778093E800A1D38FE18093E1
:101F1000200119C1853059F4809132018B3009F0CC
:101F20000DC18091E800877F8093E8002EC0882350
:101F300009F004C180913101803A71F5809132013C
:101F4000882309F0FBC08091330190913401892BE3
:101F500009F0F4C08091350190913601892B09F088
:101F6000EDC08091370190913801049709F0E6C0E7
:101F70008091E800877F8093E8001092F100109232
:101F8000F1001092F1001092F1008091E8008E773C
:101F90008093E8005CD3D7C0833AB1F580913201D9
:101FA000882309F0CBC08091330190913401892BB3
:101FB00009F0C4C08091370190913801049709F06D
:101FC000BDC0E09135018E2F8150863008F0BBC036
:101FD0008091E800877F8093E800F0E03197EE0F72
:101FE000FF1FDF01A050BF4F8C9111969C918093F1
:101FF000F1009093F100EC5EFE4F8081918180931F
:10200000F1009093F100C1CF833209F097C0809125
:102010003201833009F048C0809137019091380136
:10202000892B09F041C010913501812F81508630F4
:1020300008F089C08091E800877F8093E800809154
:10204000E8008E778093E80002D38091330190916D
:1020500034018430910591F0089709F074C016306E
:1020600009F071C080912001882309F06CC082E0E2
:10207000809320018FE08093270165C0E12FF0E07D
:1020800081E090E0012E02C0880F991F0A94E2F7C8
:1020900080932101EE0FFF1FEE5EFE4F8081918144
:1020A0008061918380834FC080913201813009F03B
:1020B00045C08091370190913801892B09F03EC0CD
:1020C00010913501812F8150863008F03CC08091FD
:1020D000E800877F8093E8008091E8008E77809306
:1020E000E800B5D28091330190913401803191059F
:1020F00019F0449741F511C0212F30E0F901EE0F9E
:10210000FF1FEE5EFE4F808191818E7F91838083E1
:10211000309324012093230116C0212F30E0F901D0
:10212000EE0FFF1FEE5EFE4F808191818F7E9183C7
:102130008083309326012093250105C080E490E040
:1021400060E070E06ADD1F91089582E08093E9000D
:102150008091E80085FF1CC088E090E060E070E0BE
:102160007CD58091E8008B778093E80080912A01EC
:1021700090912B01089690932B0180932A01803433
:10218000910534F083E18093200182E3809327015D
:1021900081E08093E9008091E80085FF2DC0809167
:1021A0002001833149F580912701882329F5809109
:1021B00028019091290180349105F4F4835F944EB5
:1021C00068E070E040E050E007D58091E8008E774D
:1021D0008093E800809128019091290108969093BE
:1021E0002901809328018034910534F084E18093A3
:1021F00020018FE080932701089584B7877F84BFF3
:1022000088E10FB6F89480936000109260000FBED2
:1022100080E090E020E80FB6F8942093610080936E
:1022200061000FBE83E08093810081E080936F00A6
:10223000569A5E9A9DD2789408952F923F924F922B
:102240005F926F927F928F929F92AF92BF92CF9246
:10225000DF92EF92FF920F931F93CFDF5E98109261
:10226000200180E0A2DCF7E02F2E0FE0E1E17E2EDE
:1022700072E1672E65E1562E56E1452E4DE2342E71
:1022800037E1C32E28E1B22E14E199E1A92E8AE1AB
:10229000982EBBE18B2EACE1FA2EFDE1EF2EEEE1A4
:1022A000DE2E80911301882309F4D9DC809113017B
:1022B000853009F44ADFFFD480912001823051F447
:1022C00080912701882331F481E090E0E8DC83E00D
:1022D0008093200180912001833059F48091250161
:1022E00090912601019729F481E05FDC84E08093DE
:1022F000200180912001853059F4809127018823A5
:1023000039F453DC82E090E0CADC86E0809320015F
:1023100080912001863051F4809125019091260111
:10232000029721F482E041DC20922001809120017B
:10233000883059F480912701882339F436DC83E012
:1023400090E0ADDC89E0809320018091200189300C
:1023500059F48091250190912601039729F483E097
:1023600024DC8AE080932001809120018B3059F495
:1023700080912701882339F418DC82E090E0AEDCFC
:102380008CE080932001809120018C3059F4809161
:10239000230190912401029729F48DE0809320017C
:1023A00000932701809120018D3051F48091270105
:1023B000882331F484E090E072DC8EE08093200189
:1023C000809120018E3051F4809125019091260159
:1023D000049721F484E0E9DB00932001809120013F
:1023E000803169F480912701882349F4DEDB81E0A4
:1023F0008093220185E090E052DC70922001809170
:102400002001813151F48091250190912601059799
:1024100021F485E0CADB60922001809120018431A3
:1024200069F480912701882349F4BFDB81E0809320
:10243000220183E090E052DC509220018091200143
:10244000853151F48091230190912401039721F467
:10245000409220013092270180912001863151F471
:1024600080912701882331F4A0DB85E090E036DC01
:10247000C092200180912001873151F48091230185
:1024800090912401059721F4B09220011093270127
:1024900080912001883151F480912701882331F403
:1024A00084DB84E090E01ADCA0922001809120017E
:1024B000893151F48091230190912401049721F4F2
:1024C0009092200110932701809120018A3151F4CC
:1024D00080912701882331F468DB81E090E0FEDB06
:1024E00080922001809120018B3151F48091230151
:1024F00090912401019721F4F0922001109327017B
:10250000809120018C3151F480912701882331F48E
:102510004CDB86E090E0C3DBE0922001809120015B
:102520008D3151F48091250190912601069721F477
:1025300086E03BDBD0922001809120018F3109F0B1
:10254000B0CE5E9AAECE1F93DF93CF93CDB7DEB7FA
:102550002A970FB6F894DEBF0FBECDBF182F742F89
:102560009E012F5F3F4FFE013696D901AF018A2FA2
:10257000821B8093E9008091EC008D938091ED00A7
:102580008193A417B50799F7812F90E0FE01E80F1A
:10259000F91F6183A80FB91F7C9391E09093E90024
:1025A0001092F0001092E8001092ED008091EB0084
:1025B0008E7F8093EB009F5F953081F720E030E0C5
:1025C000BE016A5F7F4FAE014F5F5F4FFB01E20FBD
:1025D000F31F908191FF15C02093E9008091EB00DB
:1025E00081608093EB00FA01E20FF31F80818093FA
:1025F000EC009093ED008091EE0087FD02C080E03A
:1026000008C02F5F3F4F2530310501F71093E900D7
:1026100081E02A960FB6F894DEBF0FBECDBFCF91F2
:10262000DF911F9108951092F40090E09093E900DB
:102630001092F0001092E8001092ED008091EB00F3
:102640008E7F8093EB009F5F953081F70895809196
:10265000310188239CF404C0809130018823B9F0B3
:102660008091E80082FFF8CF8091E8008B7780931B
:10267000E800089580913001882349F08091E800B6
:1026800080FFF8CF8091E8008E778093E80008956E
:1026900094E68091EC0080FF05C08091E80080FF07
:1026A00005C025C08091E80082FD21C080913001E5
:1026B000882311F482E0089580913001853011F46F
:1026C00083E008958091EB0085FF02C081E00895CA
:1026D0008091E10082FFDDCF8091E1008B7F8093CC
:1026E000E100992311F484E008959150D2CF80E065
:1026F000089543D045D01092300110922E011092CF
:102700002D0110922C0184E089BD89B5826089BDBC
:1027100009B400FEFDCF8091D800982F9F77909349
:10272000D80080688093D800809163008E7F80936A
:1027300063008091D8008F7D8093D8008091E00065
:102740008E7F8093E0008091E1008E7F8093E10096
:102750008091E20081608093E2008091E100877FB8
:102760008093E1008091E20088608093E200089508
:10277000C0DF81E080932F0108951092E200089558
:102780001092E10008951F920F920FB60F9211243C
:102790002F933F934F935F936F937F938F939F9369
:1027A000AF93BF93EF93FF938091E10080FF1CC034
:1027B0008091E20080FF18C08091E1008E7F8093BD
:1027C000E1008091E2008E7F8093E2008091E20040
:1027D00080618093E2008091D80080628093D8006D
:1027E00019BC1092300163DB8091E10084FF2AC0A4
:1027F0008091E20084FF26C084E089BD89B58260B3
:1028000089BD09B400FEFDCF8091D8008F7D8093F3
:10281000D8008091E1008F7E8093E1008091E200FA
:102820008F7E8093E2008091E20081608093E200DD
:1028300080912E01882311F481E001C084E080930F
:10284000300134DB8091E10083FF23C08091E200FE
:1028500083FF1FC08091E100877F8093E10082E0C9
:102860008093300110922E018091E1008E7F809341
:10287000E1008091E2008E7F8093E2008091E2008F
:1028800080618093E200CFDE80E060E042E05BDECA
:102890000FDB8091E10082FF0AC08091E20082FF9D
:1028A00006C08091E1008B7F8093E10002DBFF9105
:1028B000EF91BF91AF919F918F917F916F915F91B8
:1028C0004F913F912F910F900FBE0F901F90189531
:1028D0001F93DF93CF9300D0CDB7DEB7E1E3F1E0F4
:1028E0008091F100819381E0E933F807C9F7809185
:1028F000310130913201353009F487C0363040F46F
:102900003130C9F1313070F0333009F0F1C033C0EB
:10291000383009F4B5C0393009F4C4C0363009F094
:10292000E7C092C0803821F0823809F0E1C008C0C9
:1029300080912D01882311F093E013C091E011C024
:102940008091350187708093E9008091EB0090E0E1
:1029500025E0969587952A95E1F7982F917010922A
:10296000E9008091E800877F8093E8009093F10070
:102970001092F10090C0882319F0823009F0B8C09D
:1029800090E08F719070009721F0029709F0B1C02C
:102990000CC080913301813009F0ABC010922D0141
:1029A000333069F580932D012AC08091330188234B
:1029B00031F520913501277009F49BC02093E9007F
:1029C0008091EB0080FF95C0333021F48091EB00C3
:1029D000806213C08091EB0080618093EB0081E006
:1029E00090E002C0880F991F2A95E2F78093EA00D1
:1029F0001092EA008091EB0088608093EB001092C7
:102A0000E9008091E800877F49C0882309F070C001
:102A1000109133018091E800877F8093E80017DEF2
:102A200005C080913001882309F463C08091E800DB
:102A300080FFF7CF812F8F7711F492E001C093E0F0
:102A400090933001A2D855C0809133019091340108
:102A500060913501AE014F5F5F4F5FD9BC010097B8
:102A600009F447C08091E800877F8093E80089815E
:102A70009A8153D08091E8008B778093E80039C029
:102A80008038B1F58091E800877F8093E8008091DD
:102A90002E018093F1008091E8008E778093E8000A
:102AA000D6DD27C0882321F580E091E060E0AE010B
:102AB0004F5F5F4F32D9892BE1F090913301E9816B
:102AC000FA817196E491E917A0F08091E800877F80
:102AD0008093E80090932E01BADD80912E01882327
:102AE00011F483E001C084E080933001E3D901C098
:102AF000F8D98091E80083FF0AC08091EB008062E2
:102B00008093EB008091E800877F8093E8000F902E
:102B10000F90CF91DF911F9108959C014091370153
:102B2000509138014617570710F490E03DC06115E9
:102B3000710511F0AB01F9CF8091E8008E77809399
:102B4000E80040E050E0F1CF8091E80083FF02C050
:102B500081E008958091E80082FD34C080913001C9
:102B60008823B1F1809130018530A1F18091E80096
:102B700080FF1AC08091F20009C0F9012F5F3F4F1A
:102B8000E491E093F100415050408F5F41155105B1
:102B900011F0883090F390E0883009F491E0809152
:102BA000E8008E778093E8004115510569F6992376
:102BB00059F608C080913001882351F0809130018E
:102BC000853041F08091E80082FFF4CF80E00895E5
:102BD00082E0089583E00895BF92CF92DF92EF9252
:102BE000FF920F931F93CF93DF93F82EE92E8B0163
:102BF0006A014EDDB82E882329F58F2D9E2D9C016C
:102C0000E9011DC08091E80085FD12C08091E800B7
:102C10008E778093E800C114D10431F0F601099554
:102C2000813011F485E00FC033DD882341F00BC003
:102C3000FE012196E491E093F1000150104001154E
:102C4000110501F78B2DDF91CF911F910F91FF900F
:102C5000EF90DF90CF90BF900895FF920F931F9356
:102C6000CF93DF93EC018B0113DDF82E8823D1F095
:102C70001BC08091E80085FD12C08091E8008B7731
:102C80008093E8000115110531F0F80109958130B4
:102C900011F485E00AC0FCDC882321F006C0809195
:102CA000F1002197209729F78F2DDF91CF911F9168
:102CB0000F91FF9008951F9380913001882361F058
:102CC0001091E9001092E9008091E80083FF01C0B3
:102CD000FFDD17701093E9001F910895F894FFCF5E
:102CE000000100010001000100010001FFFFFFFFE2
:042CF000FFFFFFFFE4
:00000001FF
